:020000040000FA
:0408000083EF09F089
:1008100003B28CEF05F0F2B4AAEF05F09EB0B2EF90
:1008200005F09EB2BAEF05F0F2A81AEF04F0F2B2AA
:100830003AEF04F09EB61FEF04F032EF09F09E96F7
:1008400000011550000A0AE000011550010A0AE0F3
:1008500000011550020A0AE032EF09F0B1EC21F074
:1008600032EF09F0A9EC23F032EF09F08BEC24F021
:1008700032EF09F0CD90F2929EA044EF04F0010116
:10088000533F44EF04F0542BB2C1B6F1B3C1B7F1FA
:10089000B4C1B8F1B5C1B9F1AEC1B2F1AFC1B3F1F4
:1008A000B0C1B4F1B1C1B5F1AAC1AEF1ABC1AFF104
:1008B000ACC1B0F1ADC1B1F1A6C1AAF1A7C1ABF114
:1008C000A8C1ACF1A9C1ADF1A2C1A6F1A3C1A7F124
:1008D000A4C1A8F1A5C1A9F19EC1A2F19FC1A3F134
:1008E000A0C1A4F1A1C1A5F19AC19EF19BC19FF144
:1008F0009CC1A0F19DC1A1F1CECF9AF1CFCF9BF1C8
:1009000053C19CF154C19DF1CF6ACE6A0101536B72
:10091000546B9E90CD800FBC0F8E0FBA93EF04F0F6
:100920000F8A32EF09F013880F8C0FBED0EF04F05E
:100930009AC19EF19BC19FF19CC1A0F19DC1A1F103
:100940009EC1A2F19FC1A3F1A0C1A4F1A1C1A5F1D3
:10095000A2C1A6F1A3C1A7F1A4C1A8F1A5C1A9F1A3
:10096000A6C1AAF1A7C1ABF1A8C1ACF1A9C1ADF173
:10097000AAC1AEF1ABC1AFF1ACC1B0F1ADC1B1F143
:10098000AEC1B2F1AFC1B3F1B0C1B4F1B1C1B5F113
:10099000B2C1B6F1B3C1B7F1B4C1B8F1B5C1B9F1E3
:1009A00001015E6B5F6B606B616B9A515E279B51BF
:1009B0005F239C5160239D5161239E515E279F516F
:1009C0005F23A0516023A1516123A2515E27A3514F
:1009D0005F23A4516023A5516123A6515E27A7512F
:1009E0005F23A8516023A9516123AA515E27AB510F
:1009F0005F23AC516023AD516123AE515E27AF51EF
:100A00005F23B0516023B1516123B2515E27B351CE
:100A10005F23B4516023B5516123B6515E27B751AE
:100A20005F23B8516023B9516123D890010161332C
:100A300060335F335E33D8900101613360335F33DD
:100A40005E33D8900101613360335F335E3300C1A0
:100A50000CF101C10DF102C10EF103C10FF104C18E
:100A600010F105C111F106C112F107C113F108C15E
:100A700014F109C115F10AC116F10BC117F134C106
:100A800035F111B84FEF05F00101620E046F010E50
:100A9000056F000E066F000E076F58EF05F001019D
:100AA000A70E046F020E056F000E066F000E076F93
:100AB0005EC100F15FC101F160C102F161C103F1EA
:100AC00048EC20F003BF04D01ABE02D01AA0108C4C
:100AD00011A070EF05F010BA70EF05F00F80108ACA
:100AE0000CC100F10DC101F10EC102F10FC103F102
:100AF00010C104F111C105F112C106F113C107F1D2
:100B000014C108F115C109F116C10AF117C10BF1A1
:100B100035C134F132EF09F00392ABB2AB98AB8838
:100B2000030103EE00F080517F0BE92604C0EFFFC4
:100B3000802B8151805D700BD8A48B820000805186
:100B4000815D700BD8A48B9281518019D8B4079025
:100B500032EF09F0F2940101453F32EF09F0462BE4
:100B600032EF09F09E900101533F32EF09F0542B10
:100B700032EF09F09E9211B82FEF07F08BB4C8EF57
:100B800005F010ACC8EF05F08B84109CC9EF05F0A0
:100B90008B94C3CF55F1C4CF56F1C28207B438EF5E
:100BA00006F047C14BF148C14CF149C14DF14AC172
:100BB0004EF15EC162F15FC163F160C164F161C178
:100BC00065F113A8E6EF05F0138C13989AC1BAF1FA
:100BD0009BC1BBF19CC1BCF19DC1BDF19EC1BEF1E9
:100BE0009FC1BFF1A0C1C0F1A1C1C1F1A2C1C2F1B9
:100BF000A3C1C3F1A4C1C4F1A5C1C5F1A6C1C6F189
:100C0000A7C1C7F1A8C1C8F1A9C1C9F1AAC1CAF158
:100C1000ABC1CBF1ACC1CCF1ADC1CDF1AEC1CEF128
:100C2000AFC1CFF1B0C1D0F1B1C1D1F1B2C1D2F1F8
:100C3000B3C1D3F1B4C1D4F1B5C1D5F1B6C1D6F1C8
:100C4000B7C1D7F1B8C1D8F1B9C1D9F10101555136
:100C50005B2756515C23E86A5D230E2E38EF06F0C1
:100C60005CC157F15DC158F15B6B5C6B5D6B078ECE
:100C70000201002F32EF09F03C0E006F1B50E00B19
:100C8000E00AE866128819BE02D019B4108E00C1BD
:100C90000CF101C10DF102C10EF103C10FF104C14C
:100CA00010F105C111F106C112F107C113F108C11C
:100CB00014F109C115F10AC116F10BC117F134C1C4
:100CC00035F101018E676CEF06F08F676CEF06F06F
:100CD00090676CEF06F0916770EF06F0A0EF06F0FA
:100CE00092C100F193C101F194C102F195C103F1E8
:100CF0000101010E046F000E056F000E066F000E5D
:100D0000076F48EC20F000C192F101C193F102C1DC
:100D100094F103C195F1006795EF06F0016795EF37
:100D200006F0026795EF06F00367A0EF06F08EC1AC
:100D300092F18FC193F190C194F191C195F10F801F
:100D4000D57ED5BE6ED0D6CF47F1D7CF48F145C1BD
:100D500049F1E86AE8CF4AF1138A1ABE02D01AA014
:100D6000108C109047C100F148C101F149C102F156
:100D70004AC103F101010A0E046F000E056F000E57
:100D8000066F000E076F48EC20F003AF10800101E2
:100D900054A7D7EF06F00F9A0F9C0F9E0101000E8B
:100DA0005E6F600E5F6F3D0E606F080E616F010138
:100DB00047BFE7EF06F04867E7EF06F04967E7EF60
:100DC00006F04A67E7EF06F0F2880CEF07F0F298BA
:100DD0005E6B5F6B606B616B9A6B9B6B9C6B9D6BCF
:100DE0009E6B9F6BA06BA16BA26BA36BA46BA56B9F
:100DF000A66BA76BA86BA96BAA6BAB6BAC6BAD6B4F
:100E0000AE6BAF6BB06BB16BB26BB36BB46BB56BFE
:100E1000B66BB76BB86BB96BD76AD66A0101456B15
:100E2000466B0CC100F10DC101F10EC102F10FC101
:100E300003F110C104F111C105F112C106F113C192
:100E400007F114C108F115C109F116C10AF117C162
:100E50000BF135C134F132EF09F032EF09F0020144
:100E6000002F89EF08F0D59ED6CF47F1D7CF48F1B4
:100E700045C149F1E86AE8CF4AF1138AD76AD66AD0
:100E80000101456B466BD58E1B50E00BE00AE8660E
:100E9000128819BE02D019B4108E18AE1D8C00C174
:100EA0000CF101C10DF102C10EF103C10FF104C13A
:100EB00010F105C111F106C112F107C113F108C10A
:100EC00014F109C115F10AC116F10BC117F134C1B2
:100ED00035F10FA0109A11B879EF07F00101620EF9
:100EE000046F010E056F000E066F000E076F82EF94
:100EF00007F00101A70E046F020E056F000E066FCA
:100F0000000E076F47C100F148C101F149C102F16C
:100F10004AC103F148EC20F003BF95EF07F01ABE79
:100F200002D01AA0108C11B00F800CC100F10DC1BD
:100F300001F10EC102F10FC103F110C104F111C1A1
:100F400005F112C106F113C107F114C108F115C171
:100F500009F116C10AF117C10BF135C134F10201D3
:100F60003C0E006F00C10CF101C10DF102C10EF188
:100F700003C10FF104C110F105C111F106C112F155
:100F800007C113F108C114F109C115F10AC116F125
:100F90000BC117F134C135F101018E67D7EF07F0AE
:100FA0008F67D7EF07F09067D7EF07F09167DBEF18
:100FB00007F00BEF08F092C100F193C101F194C169
:100FC00002F195C103F10101010E046F000E056FDE
:100FD000000E066F000E076F48EC20F000C192F182
:100FE00001C193F102C194F103C195F1006700EFD3
:100FF00008F0016700EF08F0026700EF08F00367F0
:101000000BEF08F08EC192F18FC193F190C194F172
:1010100091C195F10F80109047C100F148C101F1D5
:1010200049C102F14AC103F101010A0E046F000E29
:10103000056F000E066F000E076F48EC20F003AF3F
:101040001080010154A731EF08F00F9A0F9C0F9EFA
:101050000101000E5E6F600E5F6F3D0E606F080E47
:10106000616F47C100F148C101F149C102F14AC1B4
:1010700003F10101140E046F050E056F000E066FDB
:10108000000E076F48EC20F003AF4AEF08F0F2883B
:101090006FEF08F0F2985E6B5F6B606B616B9A6B41
:1010A0009B6B9C6B9D6B9E6B9F6BA06BA16BA26BF4
:1010B000A36BA46BA56BA66BA76BA86BA96BAA6BA4
:1010C000AB6BAC6BAD6BAE6BAF6BB06BB16BB26B54
:1010D000B36BB46BB56BB66BB76BB86BB96B0CC15C
:1010E00000F10DC101F10EC102F10FC103F110C1F8
:1010F00004F111C105F112C106F113C107F114C1C8
:1011000008F115C109F116C10AF117C10BF135C17A
:1011100034F168EC24F01E6629D01DAE11D01D9E5E
:101120001E8E19AE07D0156A040E166E176AB1EC42
:1011300021F01CD0156A166A176AB1EC21F016D09E
:101140001DAC09D01D9C1E8C010E156E166A176A07
:10115000A9EC23F00BD01DAA09D01D9A1E8A020EFD
:10116000156E166A176A8BEC24F000D08BB4C0EFB2
:1011700008F010ACC0EF08F08B84109CC1EF08F0B1
:101180008B94C3CF55F1C4CF56F1C28207B430EF70
:1011900009F047C14BF148C14CF149C14DF14AC179
:1011A0004EF15EC162F15FC163F160C164F161C182
:1011B00065F113A8DEEF08F0138C13989AC1BAF109
:1011C0009BC1BBF19CC1BCF19DC1BDF19EC1BEF1F3
:1011D0009FC1BFF1A0C1C0F1A1C1C1F1A2C1C2F1C3
:1011E000A3C1C3F1A4C1C4F1A5C1C5F1A6C1C6F193
:1011F000A7C1C7F1A8C1C8F1A9C1C9F1AAC1CAF163
:10120000ABC1CBF1ACC1CCF1ADC1CDF1AEC1CEF132
:10121000AFC1CFF1B0C1D0F1B1C1D1F1B2C1D2F102
:10122000B3C1D3F1B4C1D4F1B5C1D5F1B6C1D6F1D2
:10123000B7C1D7F1B8C1D8F1B9C1D9F10101555140
:101240005B2756515C23E86A5D230E2E30EF09F0D0
:101250005CC157F15DC158F15B6B5C6B5D6B078ED8
:1012600032EF09F002C0E0FF005001C0D8FF1000CB
:10127000A6B238EF09F00CC0A9FF0BC0A8FFA69ECC
:10128000A69CA684F29E550EA76EAA0EA76EA682F5
:10129000F28EA694A6B24AEF09F00C2A1200A96EAB
:1012A000A69EA69CA680A8500C2A120004012C0E13
:1012B000826F65EC0BF043EC21F00C504FEC09F021
:1012C000E8CF00F10C504FEC09F0E8CF01F101AF8D
:1012D0006FEF09F00101FF0E026FFF0E036FE6ECE6
:1012E00020F029677BEF09F00401200E826F65EC86
:1012F0000BF080EF09F004012D0E826F65EC0BF00E
:10130000F0EC1EF01200356A076A0F6A106A116A63
:10131000126A136A0F010E0EC16E860EC06E030EA6
:10132000C26E0F01896A110E926E080E8A6EF10E5E
:10133000936E8B6A980E946EF18EFC0E4FEC09F052
:10134000E8CF0BF00BA011800BA211820BA411842B
:101350000BA81188C90E4FEC09F0E8CF18F0CA0E9F
:101360004FEC09F0E8CF19F0CB0E4FEC09F0E8CFC5
:101370001AF0CC0E4FEC09F0E8CF1BF0CE0E4FEC7C
:1013800009F0E8CF14F0CD0E4FEC09F0E8CF34F0BF
:101390001D6A1E6A0E6A01015B6B5C6B5D6B576BAD
:1013A000586BF29A0101476B486B496B4A6B4B6B68
:1013B0004C6B4D6B4E6B4F6B506B516B526B456B67
:1013C000466BD76AD66A0F01280ED56EF28A9D90B9
:1013D000B00ECD6E01015E6B5F6B606B616B626B1B
:1013E000636B646B656B666B676B686B696B536B88
:1013F000546BCF6ACE6A0F9A0F9C0F9E9D80760E1B
:10140000CA6E9D8202013C0E006FCC6A160E4FEC34
:1014100009F0E8CF00F1170E4FEC09F0E8CF01F129
:10142000180E4FEC09F0E8CF02F1190E4FEC09F05D
:10143000E8CF03F1010103AF38EF0AF043EC21F0EC
:10144000160E0C6E00C10BF038EC09F0170E0C6E86
:1014500001C10BF038EC09F0180E0C6E02C10BF054
:1014600038EC09F0190E0C6E03C10BF038EC09F0E2
:1014700000C18EF101C18FF102C190F103C191F160
:1014800000C192F101C193F102C194F103C195F140
:101490001A0E4FEC09F0E8CF00F11B0E4FEC09F0EB
:1014A000E8CF01F11C0E4FEC09F0E8CF02F11D0E60
:1014B0004FEC09F0E8CF03F1010103AF8EEF0AF022
:1014C00043EC21F01A0E0C6E00C10BF038EC09F061
:1014D0001B0E0C6E01C10BF038EC09F01C0E0C6EEB
:1014E00002C10BF038EC09F01D0E0C6E03C10BF0BD
:1014F00038EC09F01A0E4FEC09F0E8CF00F11B0EA2
:101500004FEC09F0E8CF01F11C0E4FEC09F0E8CFE9
:1015100002F11D0E4FEC09F0E8CF03F100C196F186
:1015200001C197F102C198F103C199F1240EAC6E8B
:10153000900EAB6E240EAC6E080EB86E000EB06E40
:101540001F0EAF6E0401806B816B0F01900EAB6EAE
:101550000F019D8A0301806B816BC26B8B92156AB0
:10156000166A176A9D8607900001F28EF28C07B00A
:1015700099EF1DF00FB0ACEF16F010BEACEF16F007
:1015800012B8ACEF16F00301805181197F0BD8B46B
:1015900099EF1DF013EE00F081517F0BE126812BB6
:1015A000E7CFE8FFE00BD8B499EF1DF023EE82F00F
:1015B000C2513F0BD926E7CFDFFFC22BDF50780A9D
:1015C000D8A499EF1DF0078092C100F193C101F1F9
:1015D00094C102F195C103F10101040E046F000EE4
:1015E000056F000E066F000E076F48EC20F000AF8D
:1015F00003EF0BF00101030E926F000E936F000ECC
:10160000946F000E956F03018251720AD8B488EF6F
:1016100016F08251520AD8B488EF16F08251750A3A
:10162000D8B488EF16F08251680AD8B479EF0BF07D
:101630008251630AD8B453EF1AF08251690AD8B4C0
:101640002AEF13F082517A0AD8B43DEF14F0825198
:10165000490AD8B4C9EF12F08251500AD8B4D3EF76
:1016600011F08251700AD8B41BEF12F08251540A63
:10167000D8B44BEF12F08251740AD8B496EF12F03E
:101680008251410AD8B4F3EF0CF082514B0AD8B41E
:10169000F1EF0BF082516D0AD8B426EF11F08251B0
:1016A0004D0AD8B43FEF11F08251730AD8B4B8EFA5
:1016B00015F08251530AD8B41DEF16F08251590A21
:1016C000D8B477EF10F08AEF1AF0040114EE00F0AE
:1016D00080517F0BE12682C4E7FF802B12000401BA
:1016E0000D0E826F65EC0BF00A0E826F65EC0BF04D
:1016F00012000401680E826F65EC0BF004012C0EE1
:10170000826F65EC0BF043EC21F030C000F131C08A
:1017100001F10101E6EC20F02EC182F40401300E4B
:10172000822765EC0BF02FC182F40401300E822772
:1017300065EC0BF030C182F40401300E822765ECB9
:101740000BF031C182F40401300E822765EC0BF0FE
:1017500032C182F40401300E822765EC0BF033C1F4
:1017600082F40401300E822765EC0BF004012C0E8C
:10177000826F65EC0BF043EC21F032C000F133C016
:1017800001F1E6EC20F02EC182F40401300E822734
:1017900065EC0BF02FC182F40401300E822765EC5A
:1017A0000BF030C182F40401300E822765EC0BF09F
:1017B00031C182F40401300E822765EC0BF032C196
:1017C00082F40401300E822765EC0BF033C182F401
:1017D0000401300E822765EC0BF08BEC24F088EFCF
:1017E0001AF004014B0E826F65EC0BF004012C0E15
:1017F000826F65EC0BF081B802D034B630D00301B3
:101800008351430AD8B436EF0CF003018351630AC5
:10181000D8B438EF0CF003018351520AD8B43AEF30
:101820000CF003018351720AD8B43CEF0CF00301B1
:101830008351470AD8B43EEF0CF003018351670A85
:10184000D8B440EF0CF003018351540AD8B442EFEE
:101850000CF003018351740AD8B4B1EF0CF003010A
:101860008351550AD8B444EF0CF082D034807AD03A
:10187000349078D0348276D0349274D0348472D05C
:10188000349470D034866ED084C330F185C331F186
:1018900086C332F187C333F10101296B91EC21F04A
:1018A00008EC21F000C104F101C105F102C106F10B
:1018B00003C107F184EC21F0200EF86EF76AF66A96
:1018C0000900F5CF2CF10900F5CF2DF10900F5CF76
:1018D0002EF10900F5CF2FF10900F5CF30F1090005
:1018E000F5CF31F10900F5CF32F10900F5CF33F131
:1018F0000101296B91EC21F008EC21F048EC20F07B
:1019000000678AEF0CF001678AEF0CF002678AEF3C
:101910000CF0036701D025D004014E0E826F65ECF8
:101920000BF004016F0E826F65EC0BF004014D0E9D
:10193000826F65EC0BF00401610E826F65EC0BF0B9
:101940000401740E826F65EC0BF00401630E826F6C
:1019500065EC0BF00401680E826F65EC0BF088EF0C
:101960001AF03496CD0E0C6E34C00BF038EC09F042
:10197000CD0E4FEC09F0E8CF34F034B006D00401BE
:10198000630E826F65EC0BF005D00401430E826F8D
:1019900065EC0BF034B206D00401720E826F65EC78
:1019A0000BF005D00401520E826F65EC0BF034B4DD
:1019B00006D00401670E826F65EC0BF005D00401C0
:1019C000470E826F65EC0BF034B606D00401740E3E
:1019D000826F65EC0BF005D00401540E826F65EC4C
:1019E0000BF088EF1AF00401410E826F65EC0BF0EA
:1019F00003018351310AD8B497EF0FF003018351EB
:101A0000320AD8B4C7EF0EF003018351330AD8B4B9
:101A100050EF0EF003018351340AD8B440EF0DF0BB
:101A200003018351350AD8B41DEF0DF004013F0EB8
:101A3000826F65EC0BF088EF1AF004012C0E826FB8
:101A400065EC0BF003018451300AD8B430EF0DF08F
:101A500003018451310AD8B438EF0DF089EF0EF04C
:101A60008B900401300E826F65EC0BF03EEF0DF0B1
:101A70008B800401310E826F65EC0BF088EF1AF059
:101A8000CC0E4FEC09F0E8CF0BF004012C0E826F66
:101A900065EC0BF003018451310AD8B464EF0DF00A
:101AA00003018451300AD8B466EF0DF0030184516C
:101AB0004D0AD8B470EF0DF003018451540AD8B424
:101AC00077EF0DF08EEF0DF08A8401D08A940BAE83
:101AD00004D00BAC02D00BBA21D0E00E0B1218D000
:101AE0001F0E0B168539E844E00B0B1211D0E00EE7
:101AF0000B1684EC21F085C332F186C333F101016A
:101B0000296B91EC21F008EC21F000511F0B0B1216
:101B1000CC0E0C6E0BC00BF038EC09F00401340E47
:101B2000826F65EC0BF004012C0E826F65EC0BF0FC
:101B3000CC0E4FEC09F0E8CF1BF08AB406D00401BC
:101B4000300E826F65EC0BF005D00401310E826F10
:101B500065EC0BF004012C0E826F65EC0BF01B386A
:101B6000E840070BE8CF82F40401300E822765ECD1
:101B70000BF004012C0E826F65EC0BF043EC21F0AE
:101B80001B501F0BE8CF00F1E6EC20F032C182F4CD
:101B90000401300E822765EC0BF033C182F404019E
:101BA000300E822765EC0BF004012C0E826F65EC81
:101BB0000BF043EC21F02EC000F100AF0BD0FF0E74
:101BC000016FFF0E026FFF0E036F04012D0E826F77
:101BD00065EC0BF0E6EC20F031C182F40401300E2C
:101BE000822765EC0BF032C182F40401300E8227AB
:101BF00065EC0BF033C182F40401300E822765ECF2
:101C00000BF004012C0E826F65EC0BF043EC21F01D
:101C10002DC000F1E6EC20F031C182F40401300E59
:101C2000822765EC0BF032C182F40401300E82276A
:101C300065EC0BF033C182F40401300E822765ECB1
:101C40000BF004012C0E826F65EC0BF043EC21F0DD
:101C50002FC000F100AF0BD0FF0E016FFF0E026F1F
:101C6000FF0E036F04012D0E826F65EC0BF0E6ECA6
:101C700020F031C182F40401300E822765EC0BF0B4
:101C800032C182F40401300E822765EC0BF033C1BF
:101C900082F40401300E822765EC0BF088EF1AF015
:101CA000CB0E4FEC09F0E8CF0BF004012C0E826F45
:101CB00065EC0BF003018451450AD8B474EF0EF0C3
:101CC00003018451440AD8B477EF0EF00301845124
:101CD000300AD8B47AEF0EF003018451310AD8B437
:101CE0007EEF0EF089EF0EF00B9E83EF0EF00B8E61
:101CF00083EF0EF0FC0E0B1683EF0EF0FC0E0B16AE
:101D00000B8083EF0EF0CB0E0C6E0BC00BF038EC9B
:101D100009F00401330E826F65EC0BF004012C0E08
:101D2000826F65EC0BF0CB0E4FEC09F0E8CF1AF0A8
:101D30001ABEA2EF0EF00401450E826F65EC0BF0A7
:101D4000A7EF0EF00401440E826F65EC0BF0040166
:101D50002C0E826F65EC0BF00401300E826F65EC87
:101D60000BF004012C0E826F65EC0BF01AB0C0EF83
:101D70000EF00401300E826F65EC0BF0C5EF0EF033
:101D80000401310E826F65EC0BF088EF1AF0CA0E79
:101D90004FEC09F0E8CF0BF004012C0E826F65ECDC
:101DA0000BF003018451450AD8B403EF0FF003018F
:101DB0008451440AD8B406EF0FF0030184514D0A50
:101DC000D8B40FEF0FF003018451410AD8B409EFE2
:101DD0000FF003018451460AD8B40CEF0FF0030151
:101DE0008451560AD8B417EF0FF003018451500AFA
:101DF000D8B422EF0FF003018451520AD8B425EF72
:101E00000FF02EEF0FF00B9E28EF0FF00B8E28EF48
:101E10000FF00B9C28EF0FF00B8C28EF0FF0FC0E4F
:101E20000B1685C3E8FF030B0B1228EF0FF0C70E4C
:101E30000B1685C3E8FF070BE846E846E8460B1299
:101E400028EF0FF00B8428EF0FF00B9428EF0FF022
:101E5000CA0E0C6E0BC00BF038EC09F0CA0E4FEC3A
:101E600009F0E8CF19F00401320E826F65EC0BF037
:101E700004012C0E826F65EC0BF019BE47EF0FF0DA
:101E80000401450E826F65EC0BF04CEF0FF004017E
:101E9000440E826F65EC0BF004012C0E826F65EC32
:101EA0000BF019C0E8FF030BE8CF82F40401300EF9
:101EB000822765EC0BF004012C0E826F65EC0BF0B1
:101EC00019BC6AEF0FF00401410E826F65EC0BF054
:101ED0006FEF0FF00401460E826F65EC0BF004010A
:101EE0002C0E826F65EC0BF019C0E8FF380BE8424E
:101EF000E842E842E8CF82F40401300E822765EC24
:101F00000BF004012C0E826F65EC0BF019B490EF0E
:101F10000FF00401520E826F65EC0BF095EF0FF09D
:101F20000401500E826F65EC0BF088EF1AF0C90EB9
:101F30004FEC09F0E8CF0BF004012C0E826F65EC3A
:101F40000BF003018451450AD8B4B5EF0FF003013B
:101F50008451440AD8B4B8EF0FF0030184514D0AFC
:101F6000D8B4BBEF0FF0C9EF0FF00B9EC3EF0FF02B
:101F70000B8EC3EF0FF0F80E0B1685C3E8FF070BAF
:101F80000B12C3EF0FF0C90E0C6E0BC00BF038EC48
:101F900009F00401310E826F65EC0BF004012C0E88
:101FA000826F65EC0BF0C90E4FEC09F0E8CF18F02A
:101FB00018BE06D00401450E826F65EC0BF005D00B
:101FC0000401440E826F65EC0BF004012C0E826F4D
:101FD00065EC0BF018C0E8FF070BE8CF82F40401B2
:101FE000300E822765EC0BF004012C0E826F65EC3D
:101FF0000BF0078043EC21F029C0E8FF003B0043D1
:102000000043030BE6EC20F033C182F40401300EF0
:10201000822765EC0BF004012C0E826F65EC0BF04F
:1020200043EC21F029C001F1019F019D2AC000F17C
:102030000101E6EC20F02FC182F40401300E82276A
:1020400065EC0BF030C182F40401300E822765ECA0
:102050000BF031C182F40401300E822765EC0BF0E5
:1020600032C182F40401300E822765EC0BF033C1DB
:1020700082F40401300E822765EC0BF004012C0E73
:10208000826F65EC0BF043EC21F02BC001F12CC00A
:1020900000F1D89001330033D890013300330101AF
:1020A000E6EC20F02FC182F40401300E822765ECAB
:1020B0000BF030C182F40401300E822765EC0BF086
:1020C00031C182F40401300E822765EC0BF032C17D
:1020D00082F40401300E822765EC0BF033C182F4E8
:1020E0000401300E822765EC0BF088EF1AF0FC0E2D
:1020F0004FEC09F0E8CF0BF003018351520AD8B43A
:10210000AEEF10F003018351720AD8B4B1EF10F0B2
:1021100003018351500AD8B4B4EF10F00301835186
:10212000700AD8B4B7EF10F003018351550AD8B440
:10213000BAEF10F003018351750AD8B4BDEF10F067
:1021400003018351430AD8B4C6EF10F00301835151
:10215000630AD8B4C9EF10F0D2EF10F00B90CCEFB7
:1021600010F00B80CCEF10F00B92CCEF10F00B8244
:10217000CCEF10F00B94CCEF10F00B84CCEF10F000
:102180000B96CCEF10F00B86CCEF10F00B98CCEF49
:1021900010F00B88CCEF10F0FC0E0C6E0BC00BF0A7
:1021A00038EC09F00401590E826F65EC0BF01190C8
:1021B000119211941198FC0E4FEC09F0E8CF0BF03E
:1021C0000BA011800BA211820BA411840BA8118803
:1021D00011A0F2EF10F00401520E826F65EC0BF0CB
:1021E000F7EF10F00401720E826F65EC0BF011A88E
:1021F00001EF11F00401430E826F65EC0BF006EF66
:1022000011F00401630E826F65EC0BF011A210EF68
:1022100011F00401500E826F65EC0BF015EF11F018
:102220000401700E826F65EC0BF011A41FEF11F02A
:102230000401550E826F65EC0BF024EF11F00401E0
:10224000750E826F65EC0BF088EF1AF004016D0ECD
:10225000826F65EC0BF003018351300AD8B483EF31
:1022600011F003018351310AD8B496EF11F0030144
:102270008351320AD8B4A9EF11F08AEF1AF081B86D
:1022800003D034B488EF1AF004014D0E826F65EC70
:102290000BF084EC21F084C331F185C332F186C3A5
:1022A00033F10101296B91EC21F008EC21F00301DD
:1022B0008351300AD8B46BEF11F003018351310A16
:1022C000D8B473EF11F003018351320AD8B47BEF15
:1022D00011F08AEF1AF0FD0E0C6E00C10BF038EC15
:1022E00009F083EF11F0FE0E0C6E00C10BF038EC1C
:1022F00009F096EF11F0FF0E0C6E00C10BF038ECF8
:1023000009F0A9EF11F00401300E826F65EC0BF0BB
:1023100004012C0E826F65EC0BF043EC21F0FD0EF6
:102320004FEC09F0E8CF00F1BAEF11F00401310EE3
:10233000826F65EC0BF004012C0E826F65EC0BF0E4
:1023400043EC21F0FE0E4FEC09F0E8CF00F1BAEFBC
:1023500011F00401320E826F65EC0BF043EC21F0BA
:1023600004012C0E826F65EC0BF0FF0E4FEC09F0B0
:10237000E8CF00F1E6EC20F031C182F40401300E28
:10238000822765EC0BF032C182F40401300E822703
:1023900065EC0BF033C182F40401300E822765EC4A
:1023A0000BF088EF1AF081B803D034B2C9EF12F005
:1023B00083C32AF184C32BF185C32CF186C32DF18D
:1023C00087C32EF188C32FF189C330F18AC331F15D
:1023D0008BC332F18CC333F1010191EC21F008EC95
:1023E00021F0160E0C6E00C10BF038EC09F0170E40
:1023F0000C6E01C10BF038EC09F0180E0C6E02C126
:102400000BF038EC09F0190E0C6E03C10BF038EC30
:1024100009F000C18EF101C18FF102C190F103C139
:1024200091F100C192F101C193F102C194F103C194
:1024300095F1C9EF12F081B803D034B2C9EF12F0B0
:1024400083C32AF184C32BF185C32CF186C32DF1FC
:1024500087C32EF188C32FF189C330F18AC331F1CC
:102460008BC332F18CC333F1010191EC21F008EC04
:1024700021F000C18EF101C18FF102C190F103C1C1
:1024800091F100C192F101C193F102C194F103C134
:1024900095F1C9EF12F081B803D034B2C9EF12F050
:1024A00083C32AF184C32BF185C32CF186C32DF19C
:1024B00087C32EF188C32FF189C330F18AC331F16C
:1024C0008CC332F18DC333F1010191EC21F008ECA2
:1024D00021F00101000E046F000E056F010E066F62
:1024E000000E076F59EC20F01A0E0C6E00C10BF0B5
:1024F00038EC09F01B0E0C6E01C10BF038EC09F042
:102500001C0E0C6E02C10BF038EC09F01D0E0C6EA7
:1025100003C10BF038EC09F000C196F101C197F14D
:1025200002C198F103C199F1C9EF12F081B803D04B
:1025300034B2C9EF12F083C32AF184C32BF185C3EF
:102540002CF186C32DF187C32EF188C32FF189C3E7
:1025500030F18AC331F18CC332F18DC333F1010103
:1025600091EC21F008EC21F00101000E046F000E47
:10257000056F010E066F000E076F59EC20F000C1C9
:1025800096F101C197F102C198F103C199F1C9EF28
:1025900012F0160E4FEC09F0E8CF00F1170E4FECD9
:1025A00009F0E8CF01F1180E4FEC09F0E8CF02F185
:1025B000190E4FEC09F0E8CF03F1E6EC20F0A9EC9E
:1025C0001EF00401730E826F65EC0BF004012C0EFB
:1025D000826F65EC0BF08EC100F18FC101F190C1EB
:1025E00002F191C103F1E6EC20F0A9EC1EF0040128
:1025F000730E826F65EC0BF004012C0E826F65EC9C
:102600000BF01A0E4FEC09F0E8CF00F11B0E4FEC67
:1026100009F0E8CF01F11C0E4FEC09F0E8CF02F110
:102620001D0E4FEC09F0E8CF03F1A5EC1AF0040100
:102630002C0E826F65EC0BF096C100F197C101F191
:1026400098C102F199C103F1A5EC1AF06FEC0BF0FF
:102650008AEF1AF00401690E826F65EC0BF0040139
:102660002C0E826F65EC0BF00101040E006F000E62
:10267000016F000E026F000E036FE6EC20F02CC11C
:1026800082F40401300E822765EC0BF02DC182F438
:102690000401300E822765EC0BF02EC182F4040198
:1026A000300E822765EC0BF02FC182F40401300E4E
:1026B000822765EC0BF030C182F40401300E8227D2
:1026C00065EC0BF031C182F40401300E822765EC19
:1026D0000BF032C182F40401300E822765EC0BF05E
:1026E00033C182F40401300E822765EC0BF0040143
:1026F0002C0E826F65EC0BF00101030E006F000ED3
:10270000016F000E026F000E036FE6EC20F02CC18B
:1027100082F40401300E822765EC0BF02DC182F4A7
:102720000401300E822765EC0BF02EC182F4040107
:10273000300E822765EC0BF02FC182F40401300EBD
:10274000822765EC0BF030C182F40401300E822741
:1027500065EC0BF031C182F40401300E822765EC88
:102760000BF032C182F40401300E822765EC0BF0CD
:1027700033C182F40401300E822765EC0BF00401B2
:102780002C0E826F65EC0BF001013C0E006F000E09
:10279000016F000E026F000E036FE6EC20F02CC1FB
:1027A00082F40401300E822765EC0BF02DC182F417
:1027B0000401300E822765EC0BF02EC182F4040177
:1027C000300E822765EC0BF02FC182F40401300E2D
:1027D000822765EC0BF030C182F40401300E8227B1
:1027E00065EC0BF031C182F40401300E822765ECF8
:1027F0000BF032C182F40401300E822765EC0BF03D
:1028000033C182F40401300E822765EC0BF0040121
:102810002C0E826F65EC0BF0200EF86EF76AF66AEC
:1028200004010900F5CF82F465EC0BF00900F5CF47
:1028300082F465EC0BF00900F5CF82F465EC0BF047
:102840000900F5CF82F465EC0BF00900F5CF82F4B6
:1028500065EC0BF00900F5CF82F465EC0BF0090094
:10286000F5CF82F465EC0BF00900F5CF82F465EC4E
:102870000BF06FEC0BF08AEF1AF081B803D034B094
:102880008DEF14F08351630AD8A488EF1AF08451B5
:10289000610AD8A488EF1AF085516C0AD8A488EF91
:1028A0001AF08651410A42E08651440A1BE08651E3
:1028B000420AD8B4A9EF14F08651350AD8B414EFFF
:1028C0001CF08651360AD8B469EF1CF08651370ADD
:1028D000D8B4D2EF1CF08651380AD8B430EF1DF0CE
:1028E00088EF1AF00798079A04017A0E826F65EC58
:1028F0000BF00401780E826F65EC0BF00401640E9E
:10290000826F65EC0BF081A88DEF14F00401550E79
:10291000826F65EC0BF092EF14F004014C0E826FA5
:1029200065EC0BF06FEC0BF08AEF1AF00788079A52
:1029300004017A0E826F65EC0BF00401410E826F88
:1029400065EC0BF00401610E826F65EC0BF083EF18
:1029500014F00798078A04017A0E826F65EC0BF079
:102960000401420E826F65EC0BF00401610E826F70
:1029700065EC0BF083EF14F001016667C7EF14F00C
:102980006767C7EF14F06867C7EF14F0696715D081
:102990004F67D2EF14F05067D2EF14F05167D2EFC7
:1029A00014F052670AD00101000E006F000E016F93
:1029B000000E026F000E036F120011B80AD0010161
:1029C000620E046F010E056F000E066F000E076F9A
:1029D00009D00101A70E046F020E056F000E066FED
:1029E000000E076F66C100F167C101F168C102F115
:1029F00069C103F148EC20F003BF6FEF15F0119AA5
:102A0000119C0101000E046FA80E056F550E066F94
:102A1000020E076F66C100F167C101F168C102F1E2
:102A200069C103F166C18AF167C18BF168C18CF19C
:102A300069C18DF148EC20F003BF0BD00101000EFD
:102A40008A6FA80E8B6F550E8C6F020E8D6F118AD8
:102A5000119C0E0E4FEC09F0E8CF18F10F0E4FEC61
:102A600009F0E8CF19F1100E4FEC09F0E8CF1AF198
:102A7000110E4FEC09F0E8CF1BF191EC1FF08AC169
:102A800004F18BC105F18CC106F18DC107F148EC51
:102A900020F0078255EC1FF091EC1FF0079255ECE7
:102AA0001FF08AC100F18BC101F18CC102F18DC10F
:102AB00003F1079255EC1FF0CC0E046FE00E056F8A
:102AC000870E066F050E076F48EC20F000C118F165
:102AD00001C119F102C11AF103C11BF140D013AABF
:102AE00074EF15F0138E139A119C119A0101800E48
:102AF000006F1A0E016F060E026F000E036F4FC1BA
:102B000004F150C105F151C106F152C107F148EC81
:102B100020F003AF05D043EC21F0118C119A120084
:102B20000E0E4FEC09F0E8CF18F10F0E4FEC09F044
:102B3000E8CF19F1100E4FEC09F0E8CF1AF1110EA1
:102B40004FEC09F0E8CF1BF14FC100F150C101F18A
:102B500051C102F152C103F1078255EC1FF018C1B7
:102B600000F119C101F11AC102F11BC103F11200F8
:102B70000401730E826F65EC0BF004012C0E826F62
:102B800065EC0BF0078462C166F163C167F164C153
:102B900068F165C169F14BC14FF14CC150F14DC1B4
:102BA00051F14EC152F157C159F158C15AF1079430
:102BB000DEEC15F06FEC0BF08AEF1AF066C100F155
:102BC00067C101F168C102F169C103F10101E6ECDD
:102BD00020F0A9EC1EF00401630E826F65EC0BF08F
:102BE00004012C0E826F65EC0BF04FC100F150C157
:102BF00001F151C102F152C103F10101E6EC20F0F3
:102C0000A9EC1EF00401660E826F65EC0BF0040166
:102C10002C0E826F65EC0BF043EC21F059C100F1F2
:102C20005AC101F10101E6EC20F0A9EC1EF004010B
:102C3000740E826F65EC0BF0120010820401530ECB
:102C4000826F65EC0BF004012C0E826F65EC0BF0CB
:102C500083C32AF184C32BF185C32CF186C32DF1E4
:102C600087C32EF188C32FF189C330F18AC331F1B4
:102C70008BC332F18CC333F1010191EC21F008ECEC
:102C800021F000C166F101C167F102C168F103C121
:102C900069F18EC32AF18FC32BF190C32CF191C33C
:102CA0002DF192C32EF193C32FF194C330F195C34C
:102CB00031F196C332F197C333F1010191EC21F068
:102CC00008EC21F000C14FF101C150F102C151F1F6
:102CD00003C152F184EC21F099C32FF19AC330F172
:102CE0009BC331F19CC332F19DC333F1010191ECDF
:102CF00021F008EC21F000C159F101C15AF1DEECDC
:102D000015F004012C0E826F65EC0BF098EF16F0B5
:102D1000118E1AA002D01AAE108C19BE02D019A4BE
:102D2000108E03018251520A02E10F8201D00F92EC
:102D30008251750A02E1108401D010948251550A23
:102D400002E1108601D010968351310A03E113820B
:102D5000138402D01392139411A003D011A401D0B4
:102D60001084078410B216EF17F010A4FAEF16F0D3
:102D7000BAC166F1BBC167F1BCC168F1BDC169F1FF
:102D8000BEC16AF1BFC16BF1C0C16CF1C1C16DF1CF
:102D9000C2C16EF1C3C16FF1C4C170F1C5C171F19F
:102DA000C6C172F1C7C173F1C8C174F1C9C175F16F
:102DB000CAC176F1CBC177F1CCC178F1CDC179F13F
:102DC000CEC17AF1CFC17BF1D0C17CF1D1C17DF10F
:102DD000D2C17EF1D3C17FF1D4C180F1D5C181F1DF
:102DE000D6C182F1D7C183F1D8C184F1D9C185F1AF
:102DF00002EF17F062C166F163C167F164C168F167
:102E000065C169F1BAC186F1BBC187F1BCC188F166
:102E1000BDC189F14BC14FF14CC150F14DC151F1D0
:102E20004EC152F157C159F158C15AF107940FA040
:102E300038EF17F00101966725EF17F0976725EF38
:102E400017F0986725EF17F0996729EF17F038EF1B
:102E500017F0BCEC14F096C104F197C105F198C1CC
:102E600006F199C107F148EC20F003BF4EEF1AF0CC
:102E7000BCEC14F00101000E046F000E056F010E92
:102E8000066F000E076F79EC20F011A02AD011A276
:102E900028D0E6EC20F0296701D005D004012D0EE2
:102EA000826F65EC0BF030C182F40401300E822792
:102EB00065EC0BF031C182F40401300E822765EC21
:102EC0000BF032C182F40401300E822765EC0BF066
:102ED00033C182F40401300E822765EC0BF06FECF5
:102EE0000BF012A8C5D012981BC01CF01C3A1C4253
:102EF000070E1C1600011C50000AD8B404EF18F08D
:102F000000011C50010AD8B490EF17F000011C50CA
:102F1000020AD8B48EEF17F036EF18F036EF18F03B
:102F200043EC21F02BC001F12CC000F1D89001330B
:102F30000033D890013300330101630E046F000E9B
:102F4000056F000E066F000E076F79EC20F0280E5B
:102F5000046F000E056F000E066F000E076F48EC41
:102F600020F000C12EF043EC21F029C001F1019FB7
:102F7000019D2AC000F10101A40E046F000E056F2F
:102F8000000E066F000E076F79EC20F000C12DF0E7
:102F900000C104F101C105F102C106F103C107F14D
:102FA000640E006F000E016F000E026F000E036FC3
:102FB00048EC20F0050E046F000E056F000E066F42
:102FC000000E076F79EC20F000C104F101C105F19A
:102FD00002C106F103C107F143EC21F02EC000F15C
:102FE00048EC20F000C12FF02FC0E8FF050F2E5C49
:102FF00003E78A8436EF18F02FC0E8FF0A0F2E5C33
:1030000001E68A9436EF18F000C124F101C125F1E0
:1030100002C126F103C127F143EC21F049EC21F074
:103020001B501F0BE8CF00F10101640E046F000E6E
:10303000056F000E066F000E076F59EC20F024C1DB
:1030400004F125C105F126C106F127C107F148ECBD
:1030500020F003BF02D08A9401D08A8424C100F1F9
:1030600025C101F126C102F127C103F18AEF1AF04F
:1030700000C124F101C125F102C126F103C127F1EC
:1030800010AE4DD0109E00C108F101C109F102C17E
:103090000AF103C10BF1E6EC20F030C1DAF131C1E5
:1030A000DBF132C1DCF133C1DDF108C100F109C14E
:1030B00001F10AC102F10BC103F101016C0E046FB1
:1030C000070E056F000E066F000E076F48EC20F02C
:1030D00003BF04D00101550EDE6F1CD008C100F102
:1030E00009C101F10AC102F10BC103F10101A40EF2
:1030F000046F060E056F000E066F000E076F48EC9A
:1031000020F003BF04D001017F0EDE6F03D0010168
:10311000FF0EDE6F1D8E11AE4EEF1AF0119E24C110
:1031200000F125C101F126C102F127C103F111A06F
:1031300005D011A203D00FB04EEF1AF010A4A8EFE3
:1031400018F00401750E826F65EC0BF0ADEF18F00E
:103150000401720E826F65EC0BF004012C0E826F7D
:1031600065EC0BF0E6EC20F02967BCEF18F00401E9
:10317000200E826FBFEF18F004012D0E826F65ECF8
:103180000BF030C182F40401300E822765EC0BF0A5
:1031900031C182F40401300E822765EC0BF004018A
:1031A0002E0E826F65EC0BF032C182F40401300EFA
:1031B000822765EC0BF033C182F40401300E8227C4
:1031C00065EC0BF004016D0E826F65EC0BF00401F1
:1031D0002C0E826F65EC0BF04FC100F150C101F174
:1031E00051C102F152C103F10101E6EC20F0A9EC5A
:1031F0001EF00401480E826F65EC0BF004017A0E9C
:10320000826F65EC0BF004012C0E826F65EC0BF005
:1032100066C100F167C101F168C102F169C103F142
:103220000101E6EC20F0A9EC1EF00401630E826FB0
:1032300065EC0BF004012C0E826F65EC0BF066C19F
:1032400000F167C101F168C102F169C103F1010137
:103250000A0E046F000E056F000E066F000E076F5A
:1032600059EC20F0000E046F120E056F000E066F71
:10327000000E076F79EC20F0E6EC20F02AC182F412
:103280000401300E822765EC0BF02BC182F404019F
:10329000300E822765EC0BF02CC182F40401300E55
:1032A000822765EC0BF02DC182F40401300E8227D9
:1032B00065EC0BF02EC182F40401300E822765EC20
:1032C0000BF02FC182F40401300E822765EC0BF065
:1032D00030C182F40401300E822765EC0BF004014A
:1032E0002E0E826F65EC0BF031C182F40401300EBA
:1032F000822765EC0BF032C182F40401300E822784
:1033000065EC0BF033C182F40401300E822765ECCA
:103310000BF00401730E826F65EC0BF004012C0EB0
:10332000826F65EC0BF043EC21F059C100F15AC1FA
:1033300001F1B4EC1BF013A2EDEF19F004012C0E17
:10334000826F65EC0BF086C166F187C167F188C1B9
:1033500068F189C169F1BCEC14F00101000E046F41
:10336000000E056F010E066F000E076F79EC20F05E
:10337000E6EC20F02967C2EF19F00401200E826FFD
:10338000C5EF19F004012D0E826F65EC0BF030C112
:1033900082F40401300E822765EC0BF031C182F417
:1033A0000401300E822765EC0BF004012E0E826FB3
:1033B00065EC0BF032C182F40401300E822765EC1B
:1033C0000BF033C182F40401300E822765EC0BF060
:1033D00004016D0E826F65EC0BF013A414EF1AF06C
:1033E00004012C0E826F65EC0BF013AC02EF1AF0A7
:1033F0000401500E826F65EC0BF0139C1398139A26
:1034000014EF1AF013AE0FEF1AF00401460E826F9C
:1034100065EC0BF0139E1398139A14EF1AF0040145
:10342000530E826F65EC0BF00FB21AEF1AF00FA07B
:103430004CEF1AF004012C0E826F65EC0BF0200E9D
:10344000F86EF76AF66A04010900F5CF82F465ECBC
:103450000BF00900F5CF82F465EC0BF00900F5CF15
:1034600082F465EC0BF00900F5CF82F465EC0BF00B
:103470000900F5CF82F465EC0BF00900F5CF82F47A
:1034800065EC0BF00900F5CF82F465EC0BF0090058
:10349000F5CF82F465EC0BF06FEC0BF00F90109E03
:1034A00012988AEF1AF00401630E826F65EC0BF03C
:1034B00004012C0E826F65EC0BF090EC1AF0040105
:1034C0002C0E826F65EC0BF003EC1BF004012C0E4C
:1034D000826F65EC0BF07FEC1BF004012C0E826F09
:1034E00065EC0BF00101F80E006FCD0E016F660E5A
:1034F000026F030E036FA5EC1AF004012C0E826F0D
:1035000065EC0BF095EC1BF06FEC0BF08AEF1AF00A
:103510006FEC0BF00301C26B0790109299EF1DF056
:10352000D8900E0E4FEC09F0E8CF00F10F0E4FECE3
:1035300009F0E8CF01F1100E4FEC09F0E8CF02F1ED
:10354000110E4FEC09F0E8CF03F10101000E046FFA
:10355000000E056F010E066F000E076F79EC20F06C
:10356000E6EC20F02AC182F40401300E822765ECDB
:103570000BF02BC182F40401300E822765EC0BF0B6
:103580002CC182F40401300E822765EC0BF02DC1B2
:1035900082F40401300E822765EC0BF02EC182F418
:1035A0000401300E822765EC0BF02FC182F4040178
:1035B000300E822765EC0BF030C182F40401300E2E
:1035C000822765EC0BF031C182F40401300E8227B2
:1035D00065EC0BF004012E0E826F65EC0BF032C12E
:1035E00082F40401300E822765EC0BF033C182F4C3
:1035F0000401300E822765EC0BF004016D0E826F22
:1036000065EC0BF01200120E4FEC09F0E8CF00F160
:10361000130E4FEC09F0E8CF01F1140E4FEC09F056
:10362000E8CF02F1150E4FEC09F0E8CF03F10101EC
:103630000A0E046F000E056F000E066F000E076F76
:1036400059EC20F0000E046F120E056F000E066F8D
:10365000000E076F79EC20F0E6EC20F02AC182F42E
:103660000401300E822765EC0BF02BC182F40401BB
:10367000300E822765EC0BF02CC182F40401300E71
:10368000822765EC0BF02DC182F40401300E8227F5
:1036900065EC0BF02EC182F40401300E822765EC3C
:1036A0000BF02FC182F40401300E822765EC0BF081
:1036B00030C182F40401300E822765EC0BF0040166
:1036C0002E0E826F65EC0BF031C182F40401300ED6
:1036D000822765EC0BF032C182F40401300E8227A0
:1036E00065EC0BF033C182F40401300E822765ECE7
:1036F0000BF00401730E826F65EC0BF012000A0EE2
:103700004FEC09F0E8CF00F10B0E4FEC09F0E8CFD9
:1037100001F10C0E4FEC09F0E8CF02F10D0E4FEC69
:1037200009F0E8CF03F1B4EF1BF0060E4FEC09F0FF
:10373000E8CF00F1070E4FEC09F0E8CF01F1080ED9
:103740004FEC09F0E8CF02F1090E4FEC09F0E8CF99
:1037500003F1B4EF1BF0010143EC21F0078457C1E2
:1037600000F158C101F107940101E80E046F800EC9
:10377000056F000E066F000E076F59EC20F0000E6B
:10378000046F040E056F000E066F000E076F79ECD4
:1037900020F0880E046F130E056F000E066F000EEA
:1037A000076F48EC20F00A0E046F000E056F000E44
:1037B000066F000E076F79EC20F0E6EC20F00101B7
:1037C0002967E8EF1BF00401200E826FEBEF1BF07E
:1037D00004012D0E826F65EC0BF030C182F4040100
:1037E000300E822765EC0BF031C182F40401300EFB
:1037F000822765EC0BF032C182F40401300E82277F
:1038000065EC0BF004012E0E826F65EC0BF033C1FA
:1038100082F40401300E822765EC0BF00401430EA4
:10382000826F65EC0BF0120087C32AF188C32BF17D
:1038300089C32CF18AC32DF18BC32EF18CC32FF1D8
:103840008DC330F18EC331F190C332F191C333F1A6
:103850000101296B91EC21F008EC21F00101000E2F
:10386000046F000E056F010E066F000E076F59EC16
:1038700020F00E0E0C6E00C10BF038EC09F00F0EAC
:103880000C6E01C10BF038EC09F0100E0C6E02C189
:103890000BF038EC09F0110E0C6E03C10BF038EC94
:1038A00009F004017A0E826F65EC0BF004012C0E16
:1038B000826F65EC0BF00401350E826F65EC0BF046
:1038C00004012C0E826F65EC0BF090EC1AF092EF75
:1038D00014F087C32AF188C32BF189C32CF18AC362
:1038E0002DF18BC32EF18CC32FF18DC330F18EC31C
:1038F00031F190C332F191C333F10101296B91ECA5
:1039000021F008EC21F0880E046F130E056F000EF5
:10391000066F000E076F4DEC20F0000E046F040ED2
:10392000056F000E066F000E076F59EC20F00101C5
:10393000E80E046F800E056F000E066F000E076F15
:1039400079EC20F00A0E0C6E00C10BF038EC09F097
:103950000B0E0C6E01C10BF038EC09F00C0E0C6E66
:1039600002C10BF038EC09F00D0E0C6E03C10BF028
:1039700038EC09F004017A0E826F65EC0BF004015B
:103980002C0E826F65EC0BF00401360E826F65EC35
:103990000BF004012C0E826F65EC0BF07FEC1BF03A
:1039A00092EF14F087C32AF188C32BF189C32CF15D
:1039B0008AC32DF18BC32EF18CC32FF18DC330F14F
:1039C0008FC331F190C332F191C333F1010191EC16
:1039D00021F008EC21F0000E046F120E056F000EAE
:1039E000066F000E076F59EC20F001010A0E046FFC
:1039F000000E056F000E066F000E076F79EC20F0C9
:103A0000120E0C6E00C10BF038EC09F0130E0C6EA8
:103A100001C10BF038EC09F0140E0C6E02C10BF072
:103A200038EC09F0150E0C6E03C10BF038EC09F000
:103A300004017A0E826F65EC0BF004012C0E826F8C
:103A400065EC0BF00401370E826F65EC0BF004019E
:103A50002C0E826F65EC0BF003EC1BF092EF14F070
:103A600087C32AF188C32BF189C32CF18AC32DF1B6
:103A70008BC32EF18CC32FF18DC330F18EC331F186
:103A800090C332F191C333F10101296B91EC21F024
:103A900008EC21F0880E046F130E056F000E066F00
:103AA000000E076F4DEC20F0000E046F040E056F42
:103AB000000E066F000E076F59EC20F00101E80EB2
:103AC000046F800E056F000E066F000E076F79EC15
:103AD00020F0060E0C6E00C10BF038EC09F0070E5A
:103AE0000C6E01C10BF038EC09F0080E0C6E02C12F
:103AF0000BF038EC09F0090E0C6E03C10BF038EC3A
:103B000009F004017A0E826F65EC0BF004012C0EB3
:103B1000826F65EC0BF00401380E826F65EC0BF0E0
:103B200004012C0E826F65EC0BF095EC1BF092EF0C
:103B300014F081B803D034B057EF1EF007A811EF8E
:103B40001EF00101800E006F1A0E016F060E026F4B
:103B5000000E036F4BC104F14CC105F14DC106F1DC
:103B60004EC107F148EC20F003BF57EF1EF0A3EC65
:103B70001EF04BC100F14CC101F14DC102F14EC12B
:103B800003F1078255EC1FF018C104F119C105F1CA
:103B90001AC106F11BC107F1F80E006FCD0E016FBF
:103BA000660E026F030E036F48EC20F00E0E0C6ED3
:103BB00000C10BF038EC09F00F0E0C6E01C10BF0D8
:103BC00038EC09F0100E0C6E02C10BF038EC09F065
:103BD000110E0C6E03C10BF038EC09F007840101E3
:103BE00043EC21F057C100F158C101F107940A0ECE
:103BF0000C6E00C10BF038EC09F00B0E0C6E01C11D
:103C00000BF038EC09F00C0E0C6E02C10BF038EC26
:103C100009F00D0E0C6E03C10BF038EC09F057EFF4
:103C20001EF007AA57EF1EF00784010143EC21F0B4
:103C300057C100F158C101F10794060E0C6E00C186
:103C40000BF038EC09F0070E0C6E01C10BF038ECEC
:103C500009F0080E0C6E02C10BF038EC09F0090EE9
:103C60000C6E03C10BF038EC09F0078462C100F15F
:103C700063C101F164C102F165C103F10794120E41
:103C80000C6E00C10BF038EC09F0130E0C6E01C184
:103C90000BF038EC09F0140E0C6E02C10BF038EC8E
:103CA00009F0150E0C6E03C10BF038EC09F0079803
:103CB000079A0401805181197F0B0DE09EA8FED761
:103CC00014EE00F081517F0BE126E750812B0F01AC
:103CD000AD6E59EF1EF0B7EF0AF018C100F119C12F
:103CE00001F11AC102F11BC103F1000E046F000EB5
:103CF000056F010E066F000E076F79EC20F029A109
:103D000098EF1EF02051D8B498EF1EF018C100F1C2
:103D100019C101F11AC102F11BC103F1000E046FB8
:103D2000000E056F0A0E066F000E076F79EC20F08B
:103D30001200010104510013055101130651021331
:103D40000751031312000101186B196B1A6B1B6BDF
:103D500012002AC182F40401300E822765EC0BF0B8
:103D60002BC182F40401300E822765EC0BF02CC1CC
:103D700082F40401300E822765EC0BF02DC182F431
:103D80000401300E822765EC0BF02EC182F4040191
:103D9000300E822765EC0BF02FC182F40401300E47
:103DA000822765EC0BF030C182F40401300E8227CB
:103DB00065EC0BF031C182F40401300E822765EC12
:103DC0000BF032C182F40401300E822765EC0BF057
:103DD00033C182F40401300E822765EC0BF012002F
:103DE0002FC182F40401300E822765EC0BF030C144
:103DF00082F40401300E822765EC0BF031C182F4AD
:103E00000401300E822765EC0BF032C182F404010C
:103E1000300E822765EC0BF033C182F40401300EC2
:103E2000822765EC0BF01200060E1F6E060E206E48
:103E3000060E216E1F2E1AEF1FF0202E1AEF1FF014
:103E4000212E1AEF1FF08B84020E1F6E020E206EC1
:103E5000020E216E1F2E2AEF1FF0202E2AEF1FF0D8
:103E6000212E2AEF1FF08B941200FF0E206E20C02F
:103E700021F0030E1F6E8B841F2E3BEF1FF0030EED
:103E80001F6E212E3BEF1FF08B9420C021F0030EFC
:103E90001F6E1F2E49EF1FF0030E1F6E213E49EFCC
:103EA0001FF0202E37EF1FF012000101005305E133
:103EB000015303E1025301E1002B18EC20F043EC25
:103EC00021F03951006F3A51016F420E046F4B0ED1
:103ED000056F000E066F000E076F59EC20F000C151
:103EE00004F101C105F102C106F103C107F118C1D6
:103EF00000F119C101F11AC102F11BC103F107B2AE
:103F000086EF1FF04DEC20F088EF1FF048EC20F01A
:103F100000C118F101C119F102C11AF103C11BF16D
:103F2000120043EC21F059C100F15AC101F1060E13
:103F30004FEC09F0E8CF04F1070E4FEC09F0E8CFA1
:103F400005F1080E4FEC09F0E8CF06F1090E4FEC31
:103F500009F0E8CF07F148EC20F000C124F101C1DD
:103F600025F102C126F103C127F1290E046F000ECD
:103F7000056F000E066F000E076F59EC20F0EE0E75
:103F8000046F430E056F000E066F000E076F4DECB9
:103F900020F024C104F125C105F126C106F127C195
:103FA00007F159EC20F000C11CF101C11DF102C163
:103FB0001EF103C11FF1120E4FEC09F0E8CF04F11E
:103FC000130E4FEC09F0E8CF05F1140E4FEC09F099
:103FD000E8CF06F1150E4FEC09F0E8CF07F10D0E12
:103FE000006F000E016F000E026F000E036F59ECA0
:103FF00020F0180E046F000E056F000E066F000E05
:10400000076F79EC20F01CC104F11DC105F11EC140
:1040100006F11FC107F14DEC20F06A0E046F2A0E65
:10402000056F000E066F000E076F48EC20F01200BF
:10403000BF0EFA6E200E3A6F396BD89000370137F9
:1040400002370337D8B029EF20F03A2F1EEF20F0C7
:1040500039073A070353D8B412000331070B80091C
:104060003F6F03390F0B010F396F80EC5FF0406F2A
:10407000390580EC5FF0405D405F396B3F33D8B06D
:10408000392739333FA93EEF20F04051392712003C
:10409000010168EC21F0D8B01200010103510719A9
:1040A000346F2BEC21F0D8900751031934AF800FF7
:1040B00012000101346B4FEC21F0D8A065EC21F027
:1040C000D8B012003AEC21F043EC21F01F0E366F0D
:1040D0007BEC21F00B35D8B02BEC21F0D8A00335C8
:1040E000D8B01200362F68EF20F034B152EC21F036
:1040F00012000101346B045105110611071100086B
:10410000D8A04FEC21F0D8A065EC21F0D8B0120077
:10411000086B096B0A6B0B6B7BEC21F01F0E366F83
:104120007BEC21F007510B5DD8A4A3EF20F00651E2
:104130000A5DD8A4A3EF20F00551095DD8A4A3EF30
:1041400020F00451085DD8A0B6EF20F00451085FBC
:104150000551D8A0053D095F0651D8A0063D0A5F6C
:104160000751D8A0073D0B5FD8900081362F90EF04
:1041700020F034B152EC21F0346B4FEC21F0D890A8
:104180007FEC21F007510B5DD8A4D3EF20F006514E
:104190000A5DD8A4D3EF20F00551095DD8A4D3EF70
:1041A00020F00451085DD8A0E2EF20F0003FE2EFDC
:1041B00020F0013FE2EF20F0023FE2EF20F0032B7E
:1041C000D8B4120034B152EC21F012000101346B6A
:1041D0004FEC21F0D8B0120084EC21F0200E366FA5
:1041E000003701370237033711EE33F00A0E376F0D
:1041F000E7360A0EE75CD8B0E76EE552372FF8EFE6
:1042000020F0362FF0EF20F034B12981D890120041
:1042100001010A0E346F200E366F11EE29F0345171
:10422000376F0A0ED890E652D8B0E726E732372F1C
:1042300013EF21F00333023301330033362F0DEF38
:1042400021F0E750FF0FD8A00335D8B0120029B1F4
:1042500052EC21F01200045100270551D8B0053D61
:1042600001270651D8B0063D02270751D8B0073DB7
:10427000032712000051086F0151096F02510A6FA4
:1042800003510B6F12000101006B016B026B036B9A
:1042900012000101046B056B066B076B12000335FE
:1042A000D8A012000351800B001F011F021F031F23
:1042B000003F62EF21F0013F62EF21F0023F62EF29
:1042C00021F0032B342B032512000735D8A0120050
:1042D0000751800B041F051F061F071F043F78EFBF
:1042E00021F0053F78EF21F0063F78EF21F0072B12
:1042F000342B072512000037013702370337083700
:1043000009370A370B3712000101296B2A6B2B6B17
:104310002C6B2D6B2E6B2F6B306B316B326B336BC9
:10432000120001012A510F0B2A6F2B510F0B2B6F1B
:104330002C510F0B2C6F2D510F0B2D6F2E510F0B7E
:104340002E6F2F510F0B2F6F30510F0B306F3151DC
:104350000F0B316F32510F0B326F33510F0B336F25
:10436000120000011750FF0A01E11200390EC86E59
:10437000800EC76E280EC66E000EC56E1650000A5F
:10438000D8B4ECEF21F01650010AD8B405EF22F0B2
:104390001650020AD8B41EEF22F01650030AD8B401
:1043A00037EF22F01650040AD8B45FEF22F016500F
:1043B000050AD8B478EF22F01650060AD8B491EF67
:1043C00022F01650070AD8B4AAEF22F01650080AB5
:1043D000D8B4C3EF22F012001750000AD8B4E2EFAD
:1043E00022F01750010AD8B4E6EF22F01750020A63
:1043F000D8B4EAEF22F01750030AD8B4EEEF22F057
:104400001750040AD8B461EF23F01750000AD8B44B
:10441000F6EF22F01750010AD8B4FAEF22F0175045
:10442000020AD8B4FEEF22F01750030AD8B402EF04
:1044300023F01750040AD8B461EF23F01750000A94
:10444000D8B406EF23F01750010AD8B40AEF23F0CE
:104450001750020AD8B40EEF23F01750030AD8B44D
:1044600012EF23F01750040AD8B461EF23F017506D
:10447000000AD8B41FEF23F01750010AD8B423EF75
:1044800023F01750020AD8B427EF23F01750030A7D
:10449000D8B43BEF23F01750040AD8B43FEF23F011
:1044A0001750050AD8B443EF23F01750060AD8B4C2
:1044B00047EF23F01750070AD8B44AEF23F01750FC
:1044C000000AD8B44EEF23F01750010AD8B452EFC7
:1044D00023F01750020AD8B456EF23F01750030AFE
:1044E000D8B45AEF23F01750040AD8B45DEF23F084
:1044F0001750000AD8B465EF23F01750010AD8B45A
:1045000069EF23F01750020AD8B46DEF23F017506B
:10451000030AD8B471EF23F01750040AD8B461EF3E
:1045200023F01750000AD8B47BEF23F01750010A8C
:10453000D8B47FEF23F01750020AD8B483EF23F0EA
:104540001750030AD8B487EF23F01750040AD8B4E1
:1045500061EF23F01750000AD8B488EF23F017500A
:10456000010AD8B48CEF23F01750020AD8B490EFA8
:1045700023F01750030AD8B494EF23F01750040A1D
:10458000D8B461EF23F01750000AD8B495EF23F0A8
:104590001750010AD8B499EF23F01750020AD8B483
:1045A0009DEF23F01750030AD8B4A1EF23F0175062
:1045B000040AD8B4A2EF23F01750050AD8B4A5EF27
:1045C00023F012009E96C580172A1200E20EC96ED3
:1045D000172A1200770EC96E172A1200020EE86E13
:1045E0008AB4E88AE8CFC9FF172A12009E96C580D0
:1045F000172A1200E20EC96E172A1200790EC96E30
:10460000172A1200000EC96E172A12009E96C58046
:10461000172A1200E20EC96E172A12007A0EC96E0E
:10462000172A120019BC03D0DEC1E8FF04D01950CC
:10463000E844E8441F09E8CFC9FF172A12009E96F4
:10464000C580172A1200E20EC96E172A120011BA8D
:1046500003D011BC01D003D0050E166E3ED001016F
:10466000DA6737EF23F0100EC96E39EF23F0DAC1A5
:10467000C9FF172A1200DBC1C9FF172A1200DCC1CB
:10468000C9FF172A1200DDC1C9FF172A1200C5840D
:10469000172A1200FF0E176E1E9E12009E96C580EE
:1046A000172A1200E20EC96E172A1200760EC96E82
:1046B000172A1200C584172A1200FF0E176E1E9EBD
:1046C0001200C584162A176A12009E96C580172A02
:1046D0001200E20EC96E172A12007B0EC96E172A4D
:1046E000120011AA04D0230EC96E172A12001C0E44
:1046F000C96E172A12009E96C580172A1200E20E74
:10470000C96E172A12007C0EC96E172A1200E9D74B
:104710009E96C580172A1200E20EC96E172A120053
:104720007D0EC96E172A1200DCD79E96C580172A07
:104730001200E20EC96E172A12007E0EC96E172AE9
:104740001200CFD7C584172A1200FF0E176E1E9EC7
:1047500012001750FF0AD8B467EF24F0390EC86E64
:10476000800EC76E280EC66E000EC56E1650000A6B
:10477000D8B4C2EF23F01650010AD8B4D6EF23F014
:1047800067EF24F01750000AD8B414EF24F0175044
:10479000010AD8B418EF24F01750020AD8B422EF57
:1047A00024F01750030AD8B425EF24F01750000A5C
:1047B000D8B42BEF24F01750010AD8B42FEF24F00F
:1047C0001750020AD8B439EF24F01750030AD8B4AE
:1047D0003CEF24F01750040AD8B442EF24F01750ED
:1047E000050AD8B445EF24F01750060AD8B44BEFA9
:1047F00024F01750070AD8B44EEF24F01750080AD7
:10480000D8B454EF24F01750090AD8B457EF24F065
:1048100017500A0AD8B45DEF24F017500B0AD8B429
:1048200060EF24F067EF24F09E96C58066EF24F0D9
:1048300018B004D04E0EC96E66EF24F0500EC96E4B
:1048400066EF24F0C58466EF24F0162AFF0E176E7B
:10485000128067EF24F09E96C58066EF24F018B0B2
:1048600004D04F0EC96E66EF24F0510EC96E66EF8C
:1048700024F0C58666EF24F0C9CF25F0C59AC58817
:1048800066EF24F0C58666EF24F0C9CF26F0C59AFE
:10489000C58866EF24F0C58666EF24F0C9CF27F0FF
:1048A000C59AC58866EF24F0C58666EF24F0C9CFA7
:1048B00028F0C58AC58866EF24F0C58466EF24F029
:1048C000FF0E176E12861E9C67EF24F0172A120047
:1048D00012B012D012B213D012B414D012A6120019
:1048E00007B01200129625C029F026C02AF027C072
:1048F0002BF028C02CF0120012901282120012929B
:104900001284120000011750FF0A04E11294176A82
:10491000A9EC23F012001750FF0AD8B467EF24F077
:1049200015EC25F01650000AD8B499EF24F067EF83
:1049300024F01750000AD8B4D7EF24F01750010A1A
:10494000D8B4DCEF24F01750020AD8B4E0EF24F01A
:104950001750030AD8B4E4EF24F01750040AD8B46F
:10496000ECEF24F01750050AD8B4EFEF24F01750FD
:10497000060AD8B4F6EF24F01750070AD8B4F9EFB6
:1049800024F01750080AD8B400EF25F01750090A90
:10499000D8B403EF25F017500A0AD8B40AEF25F06F
:1049A00017500B0AD8B40DEF25F067EF24F09E9650
:1049B000C596C58013EF25F0520EC96E13EF25F092
:1049C000B40EC96E13EF25F0C9CF30F0306AC5863A
:1049D000C59AC58813EF25F0C58613EF25F0C9CF1A
:1049E00031F0316AC59AC58813EF25F0C58613EFFB
:1049F00025F0C9CF32F0326AC59AC58813EF25F089
:104A0000C58613EF25F0C9CF33F0336AC58AC58850
:104A100013EF25F0C58413EF25F0FF0E176E1286F5
:104A20001E9C14EF25F0172A1200390EC86E800E56
:0C4A3000C76E280EC66E000EC56E120088
:10BF0000E844F926000C160C2B0C3F0C520C640C68
:10BF1000760C860C960CA50CB30CC10CCF0CDC0C6B
:06BF2000E80CF40C000C1B
:00000001FF
